:1000000000308A00BF2A0000FF00030E8301A10018
:100010007F08A0000A08A8008A01A00E0408A20018
:100020007708A3007808A4007908A5007A08A6003C
:100030007B08A700831383128B1E20280B193328FB
:10004000220884002308F7002408F8002508F90096
:100050002608FA002708FB0028088A00210E8300E2
:10006000FF0E7F0E09008A113528B40A0319B50A5C
:1000700035081C3C03184728FF3A031D4328340861
:100080004C3C031847280130B600B501B4010B11F0
:100090008A11202800306600831686010B308312F7
:1000A00086008316061283120612831686128312A6
:1000B000861283160108C03901388100831281013C
:1000C0008B16C0308B048A11D32A0830F800000048
:1000D0000430F700F70B6A2805108316051003306B
:1000E000F700F70B71288312B70D8510031C7B28CE
:1000F00083168514831203188028831685108312B3
:100100008316051483120518872883168228F80B96
:1001100067280430F700F70B8B28051083160510AD
:10012000000085140330F700F70B94280330F70024
:10013000F70B9828051483120518A02883169B280E
:10014000F8010330F700F70BA32885187814051081
:1001500083160510831285108316851083120034D0
:100160003730840000080319C2280630F800F70170
:10017000F70BB828F80BB7287B30F700F70BBE2831
:10018000800BB5280034831685140430F700F70B74
:10019000C72805140330F700F70BCC28831285100D
:1001A000831685100430F700F70BD428831205104E
:1001B0008316051090308312B70065200130B70018
:1001C00065204030B70065208316851000000514B7
:1001D00083120518ED288316E8280430F700F70B82
:1001E000EF28000000000000831685140430F7009B
:1001F000F70BF8280A308312B700B0208316851455
:100200000430F700F70B022905140330F700F70B51
:10021000072983128510831685100430F700F70B29
:100220000F29831205108316051090308312B70032
:100230006520B70165208316851000000514831220
:100240000518242983161F290430F700F70B2629E7
:10025000000000000000831685140430F700F70B3F
:100260002F290A308312B700B0208A11D42AB10A8C
:100270003108033C031D3D29B1018A11D82A0830F9
:10028000B8007708B900831685140330F700F70B20
:1002900047290514831205184F2983164A29851802
:1002A0000314851C0310F80D0430F700F70B5629D2
:1002B0008316051083120510B80B43298316851485
:1002C0000330F700F70B62298312851039080319F0
:1002D0006C2983168510831200008316051483127F
:1002E0000518742983166F290430F700F70B762957
:1002F0000510831605100330F700F70B7D298312D4
:10030000851083168510831200343708380680392B
:10031000BA00B71F8D29B709B70AB81F9129B809C4
:10032000B80A3808F8013702031899293708F70086
:10033000A529F7010830B900B70DF70D3808770285
:100340000318F700F80DB90B9C29BA1FA929F80961
:10035000F80A000000343808F80137020318B329FE
:100360003708F700BF29F7010830B900B70DF70DBE
:10037000380877020318F700F80DB90BB6298A116F
:10038000262A831685140430F700F70BC5290514B7
:100390000330F700F70BCA298312851083168510E6
:1003A0000430F700F70BD2298312051083160510CD
:1003B00091308312B70065200130F7003F217808A3
:1003C000AE00F7013F217808AF00831685100000CA
:1003D000051483120518EE298316E9290430F70065
:1003E000F70BF0290000000000008316851404308C
:1003F000F700F70BF9298312AE1B022A2E083B3CAB
:10040000031C072A2E08803A483C031C0A2A0130A4
:10041000B3000B2AB301AE1F122AFF30AE06013023
:10042000B200132AB2012E08B7000A30B8008521A5
:100430007708A9002E08B7000A30B800852178088F
:10044000AA002F08B7000A30B800AB297708AB0024
:100450008A11D92A3108003A0319352A013A0319B9
:10046000362A033A0319402A492A492A2908AC00A6
:100470002A08AD00330B3F2A0B30AC00AD00492AEF
:100480002B08AC000630AD00330B482A0B30AC0013
:10049000492A8A11DA2A0330B702031C592A373055
:1004A000840000080319592A572A00000000800B15
:1004B000552A00348316860183122C088600831681
:1004C0000612831206163008B7004B228316061256
:1004D00083120612831686010B30831286003008C1
:1004E000B7004B228316860183122D0886008316DF
:1004F0008612831286163008B7004B2283168612A6
:1005000083128612831686010B3083128600300810
:10051000B7004B22320BA52A8316860108308312BE
:10052000860083168612831286163008B7004B2287
:100530008316861283128612831686010B3083126D
:1005400086003008B7004B22BD2A8316860107308B
:100550008312860083168612831286163008B7002F
:100560004B228316861283128612831686010B3065
:10057000831286003008B7004B228A11DE2A8401DC
:100580001F30830507309F00A901AA01AB01AC0110
:10059000AD01C830B000B101B201B301B401B50181
:1005A0000130B6004A28C328360BDA2AB6013729AB
:1005B000C1292A2AB1080319DE2A5A2AD42A63003B
:02400E006A3F07
:00000001FF
